:100000008A15582CFF3FFF3F0313831235088316D0
:100010009B009C139C131C14000000001A08831200
:10002000B6003608F0000800031383122108B5005B
:1000300004207008A0000800273003138312FB007F
:10004000FF30FA00FB0B25282828FA0B2528222848
:10005000DB30FA00FA0B2A280000000008000B3001
:1000600003138312FC00FF30FB00FF30FA00FC0B8F
:100070003A284128FB0B3D284028FA0B3D283A2816
:1000800037283330FB00FF30FA00FB0B48284B28A1
:10009000FA0B482845288830FA00FA0B4D28000052
:1000A0000000080003138312B403B4033408003CB7
:1000B00003185F28B4030000000000005628000069
:1000C000000000000800031383160514013083129A
:1000D0000505F1007108013A031D8228A10A0319E0
:1000E000A20AA10A0319A20A1420A10A0319A20A4A
:1000F0002108B50004207008A30070082006031929
:100100008228752808000313831685100030831297
:1001100085180130F1007108013A031DA328A10AD6
:100120000319A20AA10A0319A20A1420A10A031999
:10013000A20A2108B50004207008A3007008200658
:100140000319A32896280800031383160515003009
:10015000831205190130F1007108013A031DC4280A
:10016000A10A0319A20AA10A0319A20A1420A10ACA
:100170000319A20A2108B50004207008A300700822
:1001800020060319C428B728080003138316851511
:100190000030831285190130F1007108013A031D06
:1001A000E528A10A0319A20AA10A0319A20A142028
:1001B000A10A0319A20A2108B50004207008A300AF
:1001C000700820060319E528D8280800FF3003131B
:1001D0008316850000308312051A0130F100710882
:1001E000013A031D0729A10A0319A20AA10A03194A
:1001F000A20A1420A10A0319A20A2108B5000420AA
:100200007008A3007008200603190729FA280800BF
:10021000FF30031383168600013083120605F100B8
:100220007108013A031D2829A10A0319A20AA10A8B
:100230000319A20A1420A10A0319A20A2108B50071
:1002400004207008A30070082006031928291B2920
:100250000800FF30031383168600003083128618CF
:100260000130F1007108013A031D4A29A10A03195E
:10027000A20AA10A0319A20A1420A10A0319A20AB8
:100280002108B50004207008A30070082006031997
:100290004A293D2908000313831603138316061504
:1002A0000030831206190130F1007108013A031D74
:1002B0006D29A10A0319A20AA10A0319A20A14208E
:1002C000A10A0319A20A2108B50004207008A3009E
:1002D0007008200603196D2960290800031383168E
:1002E00086150030831286190130F1007108013A39
:1002F000031D8E29A10A0319A20AA10A0319A20A41
:100300001420A10A0319A20A2108B50004207008CC
:10031000A3007008200603198E2981290800031301
:100320008316061600308312061A0130F100710898
:10033000013A031DAF29A10A0319A20AA10A031950
:10034000A20A1420A10A0319A20A2108B500042058
:100350007008A300700820060319AF29A22908001D
:1003600003138316861600308312861A0130F100BB
:100370007108013A031DD029A10A0319A20AA10A92
:100380000319A20A1420A10A0319A20A2108B50020
:1003900004207008A300700820060319D029C3297F
:1003A000080003138316061700308312061B013062
:1003B000F1007108013A031DF129A10A0319A20AEB
:1003C000A10A0319A20A1420A10A0319A20A2108EA
:1003D000B50004207008A300700820060319F12955
:1003E000E429080003138316861700308312861B46
:1003F0000130F1007108013A031D122AA10A031904
:10040000A20AA10A0319A20A1420A10A0319A20A26
:100410002108B50004207008A30070082006031905
:10042000122A052A080003138316051083120510EB
:100430001C2001300505F1007108013A031D232A33
:10044000A10A0319A20A08000313831685100030BD
:10045000831285180130F1007108013A031D332A17
:10046000A10A0319A20A080003138316051100301C
:10047000831205190130F1007108013A031D432A66
:10048000A10A0319A20A080003138316851100307C
:10049000831285190130F1007108013A031D532AB6
:1004A000A10A0319A20A08000313831605160030D7
:1004B0008312051A0130F1007108013A031D632A05
:1004C000A10A0319A20A08000313831606140130B7
:1004D00083120605F1007108013A031D722AA10A70
:1004E0000319A20A0800031383168614003083122E
:1004F00086180130F1007108013A031D822AA10A11
:100500000319A20A080003138316031383160611A6
:100510000030831206190130F1007108013A031D01
:10052000942AA10A0319A20A080003138316861548
:100530000030831286190130F1007108013A031D61
:10054000A42AA10A0319A20A080003138316061697
:1005500000308312061A0130F1007108013A031DC0
:10056000B42AA10A0319A20A080003138316061766
:1005700000308312061B0130F1007108013A031D9F
:10058000C42AA10A0319A20A0800031383168617B6
:1005900000308312861B0130F1007108013A031DFF
:1005A000D42AA10A0319A20A08000313831605140A
:1005B000013083120505F1007108003A031DF42A89
:1005C000A10A0319A20AA10A0319A20A1420A10A66
:1005D0000319A20A2108B50004207008A3007008BE
:1005E00020060319F42AE72A08000313831685144A
:1005F0000030831285180130F1007108003A031DA4
:10060000152BA10A0319A20AA10A0319A20A142090
:10061000A10A0319A20A2108B50004207008A3004A
:10062000700820060319152B082B080003138316E6
:1006300085140030831205190130F1007108003A69
:10064000031D362BA10A0319A20AA10A0319A20A43
:100650001420A10A0319A20A2108B5000420700879
:10066000A300700820060319362B292B080003135A
:10067000831685150030831285190130F100710849
:10068000003A031D572BA10A0319A20AA10A031954
:10069000A20A1420A10A0319A20A2108B500042005
:1006A0007008A300700820060319572B4A2B080076
:1006B000FF3003138316850000308312051A0130C2
:1006C000F1007108003A031D792BA10A0319A20A4F
:1006D000A10A0319A20A1420A10A0319A20A2108D7
:1006E000B50004207008A300700820060319792BB8
:1006F0006C2B0800FF300313831686000130831231
:100700000605F1007108003A031D9A2BA10A03198E
:10071000A20AA10A0319A20A1420A10A0319A20A13
:100720002108B50004207008A300700820060319F2
:100730009A2B8D2B08000313831686140030831226
:1007400086180130F1007108003A031DBB2BA10A85
:100750000319A20AA10A0319A20A1420A10A031963
:10076000A20A2108B50004207008A3007008200622
:100770000319BB2BAE2B0800031383160313831638
:1007800006110030831206190130F1007108003A99
:10079000031DDE2BA10A0319A20AA10A0319A20A4A
:1007A0001420A10A0319A20A2108B5000420700828
:1007B000A300700820060319DE2BD12B08000313B9
:1007C000831686150030831286190130F1007108F6
:1007D000003A031DFF2BA10A0319A20AA10A03195B
:1007E000A20A1420A10A0319A20A2108B5000420B4
:1007F0007008A300700820060319FF2BF22B0800D5
:1008000003138316061600308312061A0130F10016
:100810007108003A031D202CA10A0319A20AA10A9B
:100820000319A20A1420A10A0319A20A2108B5007B
:1008300004207008A300700820060319202C132C34
:10084000080003138316861600308312861A0130BF
:10085000F1007108003A031D412CA10A0319A20AF4
:10086000A10A0319A20A1420A10A0319A20A210845
:10087000B50004207008A300700820060319412C5D
:10088000342C080003138316061700308312061B4E
:100890000130F1007108003A031D622CA10A03190E
:1008A000A20AA10A0319A20A1420A10A0319A20A82
:1008B0002108B50004207008A30070082006031961
:1008C000622C552C08000313831686170030831200
:1008D000861B0130F1007108003A031D832CA10A28
:1008E0000319A20AA10A0319A20A1420A10A0319D2
:1008F000A20A2108B50004207008A3007008200691
:100900000319832C762C080001300313831205058C
:10091000F1007108003A031D902CA10A0319A20AE4
:10092000080000300313831285180130F1007108AC
:10093000003A031D9E2CA10A0319A20A08000030E8
:100940000313831205190130F1007108003A031DE9
:10095000AC2CA10A0319A20A080000300313831269
:1009600085190130F1007108003A031DBA2CA10A63
:100970000319A20A08000313831605160030831218
:10098000051A0130F1007108003A031DCA2CA10AB2
:100990000319A20A08000130031383120605F100AF
:1009A0007108AF008316061483122F08003A031D46
:1009B000DC2CA10A0319A20A08000313831686146B
:1009C0000030831286180130F1007108003A031DCF
:1009D000EC2CA10A0319A20A0800031383160615BA
:1009E0000030831206190130F1007108003A031D2E
:1009F000FC2CA10A0319A20A080000300313831279
:100A000086190130F1007108003A031D0A2DA10A70
:100A10000319A20A0800003003138312061A0130DA
:100A2000F1007108003A031D182DA10A0319A20A4A
:100A30000800003003138312061B0130F100710817
:100A4000003A031D262DA10A0319A20A080000304E
:100A500003138312861B0130F1007108003A031D55
:100A6000342DA10A0319A20A0800013003138312CE
:100A7000A4002408283C031C4F2D05140830FA005C
:100A8000FA0B402D0000000005100330FA00FA0BAD
:100A9000472D2408283A03194F2DA40A392D063072
:100AA000FA00FA0B512D00000800013003138312E5
:100AB000A4002408283C031C6F2D05150830FA00FB
:100AC000FA0B602D0000000005110330FA00FA0B4C
:100AD000672D2408283A03196F2DA40A592D0630D2
:100AE000FA00FA0B712D000008002F202F200800BB
:100AF000023003138312FC00FF30FB00FF30FA00CA
:100B0000FC0B832D8A2DFB0B862D892DFA0B862D50
:100B1000832D802D0630FB00FF30FA00FB0B912D5A
:100B2000942DFA0B912D8E2D0A30FA00FA0B962D8A
:100B30000000080003138312AF0CAF1325088400D4
:100B40000130B200B30133083102031DA92D320870
:100B50003002031CDC2D0130F2002608F10072087F
:100B6000F00071080319B82DF00D7010FF3FB22D81
:100B7000700880042F08B40052200130F2002608CB
:100B8000F1007208F00071080319CA2DF00D701001
:100B9000FF3FC42DF009700880052F08B4005220D3
:100BA00033083106031DD62D300832060319DC2D1B
:100BB000B20A0319B30AA32D080003138316861380
:100BC0000613831286170613080003138316861371
:100BD0000613831286130617080003138316861262
:100BE0000612831286160612080003138316861255
:100BF0000612831286120616080003138312A10A36
:100C00000319A20A2108B50004207008A7002708CC
:100C1000673A031D102E83160510831205107B2ED4
:100C20002708683A031D192E831685108312851034
:100C30007B2E2708693A031D222E83160511831285
:100C400005117B2E27086A3A031D2B2E831685116A
:100C5000831285117B2E27086B3A031D312E051256
:100C60007B2E27086C3A031D3A2E8316061083123A
:100C700006107B2E27086D3A031D432E831686101F
:100C8000831286107B2E27086E3A031D4E2E831684
:100C9000061183120611831686117B2E0313831609
:100CA000831227086F3A031D572E86117B2E2708C3
:100CB000703A031D602E83160612831206127B2ED5
:100CC0002708713A031D692E831686128312861235
:100CD0007B2E2708723A031D722E83160613831289
:100CE00006137B2E2708733A031D7B2E831686136B
:100CF000831286137B2E0313831208000230031322
:100D00008316850086013525003085180130F100F5
:100D10007108003A031D9A2E5525003085180130C0
:100D2000F1007108003A031D982E06148614992EBE
:100D30008614A72E5525003085180130F100710862
:100D4000003A031DA52E0614A72E061086100800D3
:100D50000313831205108510051185110800031374
:100D6000831686018312860108000313831205147B
:100D70008514051585150800FF30031383128600BE
:100D80000800752575252F2008001A3003138312DB
:100D9000FB00FF30FA00FB0BCE2ED12EFA0BCE2E2D
:100DA000CB2EE730FA00FA0BD32E0000000008002B
:100DB000033003138312FB00FF30FA00FB0BE12E1C
:100DC000E42EFA0BE12EDE2E9630FA00FA0BE62E18
:100DD00000000800782578250800FF3FFF3FFF3F0F
:100DE000FF3FFF3FFF3FFF3FFF3FFF3FFF3FFF3F13
:100DF000FF3FFF3FFF3FFF3FFF3FFF3FFF3FFF3F03
:100E0000FF3FFF3FFF3FFF3FFF3FFF3FFF3FFF3FF2
:100E1000FF3FFF3FFF3FFF3FFF3FFF3FFF3FFF3FE2
:101000000230031383122107F00022080318013F66
:10101000F1000030F1077008A1007108A20070080B
:10102000B5008A1104208A157008A70070082F3AAD
:10103000031D8E280130A102031CA2032108B50064
:101040008A1104208A157008A7002708673A031D33
:101050002D288A1163208A158D282708683A031DD8
:1010600035288A1183208A158D282708693A031D9F
:101070003D288A11A4208A158D2827086A3A031D65
:1010800045288A11C5208A158D2827086B3A031D2B
:101090004D288A11E6208A158D2827086C3A031DF1
:1010A00055288A1108218A158D2827086D3A031DB5
:1010B0005D288A1129218A158D2827086E3A031D7B
:1010C00065288A114B218A158D2827086F3A031D40
:1010D0006D288A116E218A158D282708703A031D04
:1010E00075288A118F218A158D282708713A031DCA
:1010F0007D288A11B0218A158D282708723A031D90
:1011000085288A11D1218A158D282708733A031D55
:101110008D288A11F2218A158D2801290130A1021A
:10112000031CA2032108B5008A1104208A15700847
:10113000A7002708673A031DA1288A1113228A15E0
:1011400001292708683A031DA9288A1124228A1533
:1011500001292708693A031DB1288A1134228A150A
:10116000012927086A3A031DB9288A1144228A15E1
:10117000012927086B3A031DC1288A1154228A15B8
:10118000012927086C3A031DC9288A1164228A158F
:10119000012927086D3A031DD1288A1173228A1567
:1011A000012927086E3A031DD9288A1183228A153E
:1011B000012927086F3A031DE1288A1195228A1513
:1011C00001292708703A031DE9288A11A5228A15EA
:1011D00001292708713A031DF1288A11B0218A15C7
:1011E00001292708723A031DF9288A11B5228A15A8
:1011F00001292708733A031D01298A11C5228A157E
:10120000012908000230031383122107F00022088D
:101210000318013FF1000030F1077008A1007108C8
:10122000A2007008B5008A1104208A157008A70072
:1012300070082F3A031D90290130A102031CA2035C
:101240002108B5008A1104208A157008A700270814
:10125000673A031D2F298A11D5228A158F2927085D
:10126000683A031D37298A11F5228A158F29270824
:10127000693A031D3F298A1116238A158F292708E9
:101280006A3A031D47298A1137238A158F292708AF
:101290006B3A031D4F298A1158238A158F29270875
:1012A0006C3A031D57298A117A238A158F2927083A
:1012B0006D3A031D5F298A119B238A158F29270800
:1012C0006E3A031D67298A11BC238A158F292708C6
:1012D0006F3A031D6F298A11DF238A158F2927088A
:1012E000703A031D77298A1100248A158F2927084F
:1012F000713A031D7F298A1121248A158F29270815
:10130000723A031D87298A1142248A158F292708DA
:10131000733A031D8F298A1163248A158F29032AA2
:101320000130A102031CA2032108B5008A11042088
:101330008A157008A7002708673A031DA3298A1198
:1013400084248A15032A2708683A031DAB298A11C9
:1013500091248A15032A2708693A031DB3298A11A3
:101360009F248A15032A27086A3A031DBB298A117C
:10137000AD248A15032A27086B3A031DC3298A1155
:10138000BB248A15032A27086C3A031DCB298A112E
:10139000CB248A15032A27086D3A031DD3298A1105
:1013A000DD248A15032A27086E3A031DDB298A11DA
:1013B000ED248A15032A27086F3A031DE3298A11B1
:1013C000FD248A15032A2708703A031DEB298A1188
:1013D0000B258A15032A2708713A031DF3298A1160
:1013E00021248A15032A2708723A031DFB298A1132
:1013F00019258A15032A2708733A031D032A8A111F
:1014000027258A15032A0800063003138312FC00DF
:10141000FF30FB00FF30FA00FC0B0F2A162AFB0BF3
:10142000122A152AFA0B122A0F2A0C2A1A30FB004C
:10143000FF30FA00FB0B1D2A202AFA0B1D2A1A2A5C
:101440004230FA00FA0B222A000008002830031369
:101450008312AF00F430B0000130B1008A119A2538
:101460008A1508000030031383128C1A0130F10032
:101470007108AB002B08F0000800031383121A0850
:10148000AB00003098180130F1007108013A031DDB
:101490004B2A181218162B08F000080003138316A5
:1014A000003003138316981801308312F10071087D
:1014B000003A031D5D2A00004E2A2B0899000800FF
:1014C000031383160030031383169C180130831214
:1014D000F1007108013A031D6F2A0000602A2B08F1
:1014E00083169B0083122C0883169A007F301C05FC
:1014F0008312F000700883169C000430831270047D
:1015000083169C008B1355309D00AA309D009C14BF
:101510008B171C1108000313831698169030831242
:101520009800831686140611003083128C1A01303D
:10153000F1007108013A0319942A080001300313DD
:101540008312A100A2012108B5008A1104208A1586
:101550007008A70070087F3A031DAF2AEE2B803079
:10156000F000803022067002031DB82A2108DC3CFE
:101570000318BB2AEE2B98132708613A031DC42ACF
:101580008A11DD258A15EA2B2708623A031DCC2A29
:101590008A11E5258A15EA2B2708633A031DD42A08
:1015A0008A11ED258A15EA2B2708643A031DDC2AE7
:1015B0008A11F5258A15EA2B2708653A031DE32AC7
:1015C000A0308600EA2B2708663A031DEA2A50302D
:1015D0008600EA2B2708673A031DF02A0514EA2B38
:1015E0002708683A031DF62A8514EA2B2708693A6A
:1015F000031DFC2A0515EA2B27086A3A031D022B56
:101600008515EA2B27086B3A031D072BEA2B2708C1
:101610006C3A031D102B8316061083120614EA2B56
:1016200027086D3A031D192B831686108312861422
:10163000EA2B27086E3A031D222B8316061183120C
:101640000615EA2B27086F3A031D2B2B83168611EC
:1016500083128615EA2B2708703A031D342B831654
:10166000061283120616EA2B2708713A031D3D2B3A
:101670008316861283128616EA2B2708723A031DF8
:10168000462B8316061383120617EA2B2708733A94
:10169000031D4F2B8316861383128617EA2B270808
:1016A000443A031D572B8A11FD258A15EA2B27087A
:1016B000463A031D5D2B0020EA2B2708473A031DFD
:1016C000632B0221EA2B2708503A031D6C2B83164B
:1016D000061483120614EA2B2708513A031D712BB6
:1016E000EA2B27084E3A031D792B8A117E268A158C
:1016F000EA2B27084D3A031D7E2BEA2B2708743A64
:10170000031D862B0130A100A201A32A2708523A0B
:10171000031D8E2B8A11A8268A15EA2B2708533A17
:10172000031D962B8A11AF268A15EA2B2708543AF7
:10173000031D9E2B8A11B5268A15EA2B2708553AD8
:10174000031DA62B8A11BC268A15EA2B2708763A98
:10175000031DAE2B8A112F208A15EA2B2708773A12
:10176000031DB62B8A1175258A15EA2B2708783AAE
:10177000031DBE2B8A11C1268A15EA2B2708793A48
:10178000031DC62B8A11C5268A15EA2B27087A3A2B
:10179000031DCE2B8A11D8268A15EA2B2708413A39
:1017A000031DD42B0422EA2B2708423A031DDC2B0D
:1017B0008A1178258A15EA2B2708433A031DE42B62
:1017C0008A11EA268A15EA2B27084F3A031DEA2BCD
:1017D0002622EA2BA10A0319A20AA32A080003134E
:1017E00083122908A50084170130F2002A08F100AD
:1017F0007208F00071080319012CF00D7010FF3F02
:10180000FB2BF009700880052A08A6000800CF30DD
:1018100003138316990018118B22A801A101A201BC
:101820008030133AF000803022067002031D1A2C1B
:101830002108883C031C4A2C32227008003A031904
:101840002F2C3D227008A9007008AB004E222808FA
:10185000AB002908AC0060228312A80A1C2C0330BC
:10186000FB00FF30FA00FB0B362C392CFA0B362C20
:10187000332C9630FA00FA0B3B2C00002208133A66
:10188000031D442C8830210603194A2CA10A031990
:10189000A20A102CA801080003138312B5018A11B3
:1018A00004208A157008213A031D572C9E22080037
:1018B0008A112F208A150530A9000330AA00EF23D2
:1018C0006430AF002C30B0000130B1008A119A258D
:1018D0008A152830AF00F430B0000130B1008A1111
:1018E0009A258A15072407309F0098131030831615
:1018F000850028308312AF005830B0000230B100AC
:101900008A119A258A158A111C208A152830AF0061
:101910002C30B0000130B1008A119A258A158A1145
:101920002F208A154C24932CFF3FFF3FFF3FFF3FA2
:02400E00623F0F
:00000001FF
